:020000040000FA
:020000001028C6
:040008008B01102830
:100020008316033086000030850083128B0183160F
:100030008F308100831217147B2081207B20903029
:100040008B007B206300C720061C5E2883160130CE
:10005000860083128614CE20CE208610940195014E
:1000600083160F3086008312950A1508031D392860
:10007000940A6400861C4728831601308600831288
:1000800086100A3090006400900B432830288316B5
:1000900001308600831214080319502817142128F0
:1000A0005A301502031C5728171485012128171CE4
:1000B0002128171081209E20812021288B01FF30CC
:1000C000850006168617C7207B20C72090308B003E
:1000D0008120812081207B20051486160617C720E9
:1000E0007B20051406168617C720C720C720C72007
:1000F000C7207B20212805100612861206138613BE
:10010000080005309000051406168617CE207B20C7
:10011000051486160617CE207B20CE20900B832850
:10012000051406160617CE20CE20CE20CE20CE20D7
:10013000051006128612061386130800053090007B
:100140007B20051486160617CE2006138617CE20B0
:1001500006178613CE2006138617CE2006178613A1
:10016000CE2006138617CE20C7207B20C720900BF9
:10017000A02808003C309600C020960BBC28080040
:1001800032309300CE206400930BC2280800053063
:100190009300CE206400930BC9280800E030910042
:0E01A00092006400920BD128910BD028080029
:02400E00F53F7C
:00000001FF
